:030000000236FCC9
:0C36FC0078FFE4F6D8FD75815E023743CC
:1014C80020000A3C2E2E2E3E004950436F6E6E655A
:1014D80063745245510A004950436F6E6E656374D8
:1014E800000A49504E6F41434B210A003E432C5697
:1014F8002C43432CC0E4E0EFF2E5F020D1E8EDEA1C
:10150800EEEC49500A003E432C4D41432C25303225
:1015180062583A25303262583A25303262583A25B4
:10152800303262583A25303262583A2530326258A1
:101538002C4D414320E0E4F0E5F10A003E432C56EF
:1015480045522C20332E3220EEF2202573202573AD
:101558002CC2E5F0F1E8FF20495020ECEEE4F3EB73
:10156800FF0A004D617920303520323031310030AA
:10157800393A32363A3436003E432C4C442C5052D9
:101588004F473A20202020202020202020202020E3
:101598002020202020202020202020202020202043
:1015A8002020202020202020202020202020202033
:1015B8002020202020202020202020202020202023
:1015C80020202020202020202CC4E0F2E020EFF072
:1015D800EEF8E8E2EAE828F4E0E9EB290A003E2A16
:1015E8002C312CCEF1EDEEE2EDFBE520EFE0F0E062
:1015F800ECE5F2F0FB20F1E5F2E5E2EEE3EE20E8BF
:10160800EDF2E5F0F4E5E9F1E00A003E412C413065
:10161800312C2562752E2562752E2562752E256260
:10162800752C495020E0E4F0E5F120E0E4E0EFF229
:10163800E5F0E00A003E412C4130322C2562752E3F
:101648002562752E2562752E2562752C495020E07D
:10165800E4F0E5F120EEF1ED2E20F1E5F0E2E5F021
:10166800E00A003E412C4130332C2562752E25625C
:10167800752E2562752E2562752C495020E0E4F000
:10168800E5F120F0E5E72E20F1E5F0E2E5F0E00AEB
:10169800003E412C4130342C2562752E2562752E72
:1016A8002562752E2562752CCCE0F1EAE020F1E583
:1016B800F2E80A003E412C4130352C2562752E2572
:1016C80062752E2562752E2562752CD8EBFEE70A09
:1016D800003E2A2C312CC4EEEF2E20EFE0F0E0EC97
:1016E800E5F2F0FB20F1E5F2E5E2EEE3EE20E8EDCD
:1016F800F2E5F0F4E5E9F1E00A003E422C5330311E
:101708002C2562752CC6E4E0F2FC20E7E0EFF0EE51
:10171800F1E020F1EEE5E4E8EDE5EDE8FF20EEF29A
:1017280020F1E5F0E2E5F0E00A003E422C533032C9
:101738002C2562752CCEE1ECE5ED20F120F1E5F0E9
:10174800E2E5F0EEEC20E1E5E720EAE2E8F2E0EDA0
:10175800F6E8E90A003E422C5330332C2562752CFA
:10176800CFE5F0E5E7E0EFF3F1EA20EFF0E820EF6E
:10177800EEF2E5F0E520F1E2FFE7E820F120F1E5FF
:10178800F0E2E5F0EEEC0A003E422C5330382C250E
:1017980062752CCCE5E4EBE5EDEDFBE92049502042
:1017A800EAE0EDE0EB28E7E0E4E5F0E6EAE020E453
:1017B800EE203520F1E5EA290A003E454E440A00AC
:1017C8000A44756D70582020202020303020303198
:1017D800203032203033203034203035203036204D
:1017E8003037203038203039203041203042203006
:1017F80043203044203045203046000A3A003A2041
:10180800000A000A44756D704420202020203030E2
:101818002030312030322030332030342030352011
:1018280030362030372030382030392030412030D1
:101838004220304320304420304520304600457255
:1018480072206B657900526420656570726F6D0A4D
:10185800005264204D454D0A00526420436F646570
:101868000A00577269746520436F64650A0044650D
:101878006275674950204F4E0A0044656275674992
:1018880050204F46460A0044656275675573657275
:10189800204F6E0A00446562756755736572204F64
:1018A80046460A0044656275674D7367204F6E0AA5
:1018B8000044656275674D7367204F46460A0043CA
:1018C8006F6E666967206C6F636B210A0057722020
:1018D800656570726F6D0A002053617665206565D5
:1018E80070726F6D210A00457272204D41432100CC
:1018F8004C6F61643E3E002A00CEF8E8E1EAE00A57
:1019080000202D202575282575290A003C413031F5
:101918003D003C4130323D003C4130333D003C41CC
:1019280030343D003C4130353D003C21003C5330D3
:10193800313D003C5330323D003C5330333D003C98
:101948005330353D003C5330383D003C5330363D34
:01195800008E
:0640EC00010B00010900B8
:10412200C28E438910758BFF758DB7D2ABD28E22AA
:03001B000235DECD
:1035DE00C0E0C083C082C0D0C28E758BFF758DB720
:1035EE0020060675A61E75A6E10509D202E50B603A
:1035FE0002050B050EE50E540F7051E50AD394012A
:10360E004002150AD20EE50E543F7012D20090669B
:10361E008EE0600A04F0E0D394B44002D2069066C5
:10362E0087E0600204F0906104E0600214F090669E
:10363E008FE0D394014003E014F0300502050CE551
:10364E000DD394644004D2068002050DE508D39490
:10365E000140021508D28ED0D0D082D083D0E03275
:1008DF00C291C290D2B5C20B7D027C007F0712403D
:1008EF00CF8F24E524646060097D017F6012406A28
:1008FF00D20BE4FDFC7F0B1240CF8F24E52430E6B2
:10090F00097D04E4FF12408ED20B7D017C007F072E
:10091F001240CF8F24E5247008FD7FFF12406AD26A
:10092F000B300B03126000C288C2A8C2AA758900DF
:10093F00123A2490633FE0B4FA06A3E064CE607BE2
:10094F00E4F52474372524F582E43463F583E4F069
:10095F000524E524B443EC90633F74FAF0A374CEFE
:10096F00F0A374CCF0906345740AF0E4A3F0A304F1
:10097F00F0A3F090633B74FFF0A3F0A3F0E4A3F0B7
:10098F009063567403F0E4F524E5242401FFE43367
:10099F00FE74372524F582E43463F583E0FD1240BD
:1009AF00460524E524C3944340DFE4F5A775A61E4E
:1009BF0075A6E1907FF0F0A3F080FE90634A740378
:1009CF00F0A374CCF0E4906349F090668CF0A3F040
:1009DF0012328BC2B5123B1CC206123ECDD20BC2D5
:1009EF000DC20C9065777408F09062B57424F0E432
:1009FF00A3F090633FE09062B7F0906340E09062A5
:100A0F00B8F0906341E09062B9F0906342E0906279
:100A1F00BAF0906343E09062BBF0906344E0906261
:100A2F00BCF0750A01E4906578F0C207C208C209EC
:100A3F00C20A200B18AF24FE7D03123371E4FF129C
:100A4F00352E7E147FC8E4FBFDFC122EA890668E17
:100A5F00E060037401F0E4906104F0F50C906576AA
:100A6F00F0F50D12412275A70775A61E75A6E1D2E6
:100A7F00AFE4F50D906104E07003120F6790668F7D
:100A8F00E06401701D9080007410F09080A874FFD6
:100A9F00F0A3F0A3F0A3F0E490668FF0D20BC20C9A
:100AAF00C20D908008E0F52430E405D2077410F0F1
:100ABF00E52430E508D2099080087420F0E5243051
:100ACF00E608D2089080087440F0E50CC394034008
:100ADF0019908002E4F0908001F0908000F0E50C16
:100AEF0094064006E4F50C123ECD9080A0E0700312
:100AFF00123C7A9080B8E07003123AA29080D0E056
:100B0F007003123E71908000E07013300710122FA7
:100B1F00AF906332EFF0D394004003120026908021
:100B2F0002E07006908000E06005D205020A80C2E4
:100B3F0005E4F50C906104E06003020A80200B12BB
:100B4F00906579E0600C7E147FCA1231A3E4906542
:100B5F0079F0300912122B1E906332EFF0D394000C
:100B6F004005E0FF124136200803020D04122997B9
:100B7F00906332EFF07003020A80906376E054BF07
:100B8F00247F7003020C5F147003020C3724026081
:100B9F0003020CA6200B077E147FD11231A3200F66
:100BAF0003020D0490634EE07006906352E060679D
:100BBF00906683E0FF90634EE0B50724906684E073
:100BCF00FE90634FE0B50618906685E0FE90635087
:100BDF00E0B5060C906686E0FE906351E06E6037DC
:100BEF00906352E06F6003020D04906684E0FF9003
:100BFF006353E06F6003020D04906685E0FF90631E
:100C0F0054E06F6003020D04906686E0FF90635519
:100C1F00E06F6003020D04C2039065787401F01257
:100C2F004139750A01020D0490668EE0600374016C
:100C3F00F090667BE0FF906378E06F6003020D0435
:100C4F0090667BE004F0E4F50A906576F0020D04FF
:100C5F00300303020D04906345E07003020A809095
:100C6F0062B4E06008906356741EF080069063567D
:100C7F007403F012001ED203E4F50A906576F0902B
:100C8F00668704F0E490667AF0A3F0200B677E1479
:100C9F007FDF1231A3805E90668EE060037401F0F7
:100CAF00300352906376E020E74B906378E0FF903B
:100CBF00667AE0FE6F600D906682E07007EE146F4B
:100CCF007033801390667AE004F0906332E0FFD3C4
:100CDF00940440031241389060007482F0A37401B1
:100CEF00F0906378E0906002F07E607F007D0312E9
:100CFF00380F020A80200303020E27E50A706E12D6
:100D0F00366EEF60237E647F76906477E02404FD77
:100D1F0012380F906682E07009906356E0F50A0270
:100D2F000A80E4F50A020A80906687E0D3943C407B
:100D3F003C906682E070369062B4E07030906687C7
:100D4F0004F0124137E4906476F0A37412F09066C9
:100D5F007BE0906478F0A374FDF090610563A201CD
:100D6F0090647A63A2017F121226E58098124132B5
:100D7F008F24E524B401159060007483F0E4A3F090
:100D8F007E607F007D0212380F020A80E524D39423
:100D9F0001401C9060007483F0A37401F0E52424DB
:100DAF00FEA3F07E607F007D0312380F020A80E5FC
:100DBF000A64016003020A80906576E004F0200B5C
:100DCF00077E147FE91231A3906576E0FFD394017B
:100DDF00400B906356E0941E5003E004F0EFC39471
:100DEF0005400DC203E4906578F0124139020A8084
:100DFF007C667D8390634AE0FAA3E0FB7F021239A1
:100E0F00A07E647F76906477E02404FD12380F9003
:100E1F006356E0F50A020A80E50A64016003020ADC
:100E2F0080906578E014604624FE604214700302DF
:100E3F000F1A24046003020A80E4F50C200F1390AC
:100E4F0065787404F0906576E05401F0750A01023C
:100E5F000A809080027410F0E4906578F0906576C7
:100E6F0004F0750A1290668374FFF0020A80906690
:100E7F0083E07003020F049064767480F0906478BE
:100E8F007401F0E4A3F0A304F0A37430F0A3747B17
:100E9F00F0E4F524747D2524F582E43464F583743D
:100EAF007DF0747E2524F582E43464F583E4F0E567
:100EBF00242407906477F07C667D8390634AE0FA80
:100ECF00A3E0FB7F021239A07E647F76E52424091C
:100EDF00FD12380F906682E0601B12001ED203E4F1
:100EEF00F50A906576F090668704F0E490667AF0E4
:100EFF00A3F0020A80300F07E4906578F080069027
:100F0F0065787404F0750A12020A809080027410DA
:100F1F00F0750A03906576E06401FFF090657874D0
:100F2F0001F0EF7019906352E06013FCA3E0FDA392
:100F3F00E0FEA3E0FF9066831222B9020A8090635D
:100F4F004EE0FCA3E0FDA3E0FEA3E0FF906683125A
:070F5F0022B9020A8080FEA6
:010F66002268
:10002600906377E0B444047F0180027F009063769A
:10003600E0B447047E0180027E00EE5F604A906372
:100046003FE0906378F0906340E0906379F09063CE
:1000560041E090637AF0906342E090637BF09063B6
:1000660043E090637CF0906344E090637DF090639E
:10007600777452F09062AE63A2019080A863A201E9
:100086007F061226E50208D5906332E0C394085035
:10009600030208DE90633FE0FF906378E06F600341
:1000A6000208DE906340E0FF906379E06F60030230
:1000B60008DE906341E0FF90637AE06F6003020818
:1000C600DE906342E0FF90637BE06F60030208DE30
:1000D600906343E0FF90637CE06F60030208DE906C
:1000E6006344E0FF90637DE06F60030208DE906387
:1000F60077E06444701A9080A8E0B4FF139062AE73
:1001060063A2019080A863A2017F061226E58010F3
:100116009062B2E09080ACF09062B3E09080ADF077
:1001260090668EE060037401F090668F7464F090C0
:1001360063777452F0906376E0646D600302027830
:100146007BFF7A1479F4121E2E7BFF7A15790E90B6
:10015600633FE0F52EA3E0F52FA3E0F530A3E0F52D
:1001660031A3E0F532A3E0F533121E2E752EFF758E
:100176002F1575306B7531FF7532157533777BFF2B
:100186007A157944121E2E7BFF7A157980121E2E5F
:100196007BFF7A1579E6121E2E7BFF7A167913906D
:1001A6006345E0F52EA3E0F52FA3E0F530A3E0F5D7
:1001B60031121E2E7BFF7A16793D90634EE0F52EA6
:1001C600A3E0F52FA3E0F530A3E0F531121E2E7B58
:1001D600FF7A16796B906352E0F52EA3E0F52FA314
:1001E600E0F530A3E0F531121E2E7BFF7A167999E1
:1001F60090633BE0F52EA3E0F52FA3E0F530A3E0F6
:10020600F531121E2E7BFF7A1679BC906337E0F526
:100216002EA3E0F52FA3E0F530A3E0F531121E2E54
:100226007BFF7A1679D9121E2E7BFF7A177902A2E6
:100236000FE433F52E121E2E7BFF7A177932906665
:1002460082E0F52E121E2E7BFF7A17795D90668E60
:10025600E0F52E121E2E7BFF7A1779909062B4E09D
:10026600F52E121E2E122D9C7BFF7A1779C2121EB6
:100276002E22906376E0644C70737E177FC8FBFD78
:10028600FC122EA890637EE0F525A3E0F526E4F5A2
:1002960028E525906380F0A3E526F07E187F037C91
:1002A600637D807B02122EA8E4F5278526828525AC
:1002B60083E0FF74802527F582E43463F583EFF04D
:1002C6000526E526700205250527E527B410DC7E00
:1002D600187F067C637D807B10122EA80528E528F2
:1002E600C3941040AC7E187F091231A32290637626
:1002F600E0646C7060F5297E187F0BFBFDFC122E06
:10030600A8E4F528E4906380F0A3E529F07E187F41
:10031600037C637D807B02122EA8E4F527A829E6DC
:10032600FF74802527F582E43463F583EFF0052911
:100336000527E527B410E67E187F067C637D807B63
:1003460010122EA80528E528C3940840B77E187F0A
:10035600091231A322906376E0644B7061F527742D
:10036600682527F582E43463F583E06032746825F6
:1003760027F582E43463F583E0F460237468252767
:10038600F582E43463F583E0FF747E2527F582E485
:100396003463F583E0B507100527E527B408C09058
:1003A60061047432F00208D59063767421F0300B44
:1003B600030208D57E187F461231A30208D5906342
:1003C60076E0B4521A200B077E187F4E1231A390A6
:1003D60063767472F07E637F767D0812378822908A
:1003E6006376E064497045200B077E187F59123109
:1003F600A390637EE0F525A3E0F526E4F5278526A0
:1004060082852583E0FF74802527F582E43463F531
:1004160083EFF00526E526700205250527E527B4B6
:1004260080DC7E637F767D8A12378822906376E051
:1004360064437046200B077E187F611231A39063D8
:100446007EE0F525A3E0F526E4F5278526828525B9
:1004560083E493FF74802527F582E43463F583EF04
:10046600F00526E526700205250527E527B480DB7D
:100476007E637F767D8A12378822906376E0645A9F
:100486007053200B077E187F6A1231A390637EE0BB
:10049600F525A3E0F5267C637D807B80AF26AE251F
:1004A600123FECE4F527852682852583E493FF74C5
:1004B600802527F582E43463F583EFF00526E526EB
:1004C600700205250527E527B480DB7E637F767DF0
:1004D6008A12378822906376E06444600302056CD2
:1004E60090637EE0FF644470030208D5EFB4310CDC
:1004F600C20B7E187F761231A30208D590637EE088
:10050600B4300CD20B7E187F821231A30208D5902C
:10051600637EE0B4320CD20C7E187F8F1231A302B8
:1005260008D590637EE0B4330CC20C7E187F9D1212
:1005360031A30208D590637EE0B4340CD20D7E1848
:100546007FAC1231A30208D590637EE0B4350CC2AD
:100556000D7E187FB91231A30208D590637EE0FFA5
:100566001241350208D5906104E07013200B077E16
:10057600187FC71231A39063767421F00208D590D4
:1005860061047432F0906376E0FFB45104C2AF8028
:10059600FEEF64577045200B077E187FD51231A3F6
:1005A60090637FE0906332F0E4F527906332E0FFDA
:1005B600E527C39F40030208D574802527F582E40A
:1005C6003463F583E0FF90637EE0252724ADF58252
:1005D600E43461F583EFF0052780D0906376E0641C
:1005E60053600302068F200B077E187FE01231A3AB
:1005F60090633FE0FF9061B6E06F703C906340E02F
:10060600FF9061B7E06F7030906341E0FF9061B892
:10061600E0B50724906342E0FF9061B9E0B50718A2
:10062600906343E0FF9061BAE0B5070C906344E045
:10063600FF9061BBE06F60169063767421F0300B1B
:10064600030208D57E187FEF1231A30208D5E4F520
:1006560027E4F50DAF27FE74AD2527F582E4346156
:10066600F583E0FD1240460527E527C394FE40E1E9
:10067600C2AFE4907FF0F0A3F0907FFD74AAF0A3E0
:1006860074FFF0A37455F080FE906376E0644F70BB
:100696005A90637EE0F525A3E0F526E5264525700C
:1006A6000A200B077E187FF81231A3200B077E184D
:1006B6007FFF1231A3E4F52774802527F582E43401
:1006C60063F583E0852682852583F00526E5267079
:1006D6000205250527E527B480DE90668DE0248097
:1006E600F090668CE03400F00208D5906376E06402
:1006F60045707490637EE0FEA3E0FF907FF0EEF01D
:10070600A3EFF0D39400EE94044038907FF0E0FE1F
:10071600A3E0FF90668CE0FCA3E0FD9FEC9E4023E7
:10072600E42FFFEE3401FED3ED9FEC9E5015C2AFD1
:10073600907FFD74AAF0A374FFF0A37455F0E4F55E
:10074600A780FE7E197F011231A37BFF7A197909F2
:10075600907FF0E0F52EA3E0F52F90668CE0F53063
:10076600A3E0F531121E2E906376E0646560030205
:1007760008DE90637EE0FFA3E0907FF0CFF0A3EF6A
:10078600F0E4F525F526D3907FF1E09526907FF0ED
:10079600E095254020E4F50D2526FFE5253401FEEC
:1007A600852682852583E0FD1240460526E52670CE
:1007B60002052580D17E197F14123896EF4E6020EF
:1007C600120003906345EFF0120003906346EFF0CA
:1007D600120003906347EFF0120003906348EFF0B6
:1007E6007E197F1A123896EF4E602012000390632E
:1007F6004EEFF012000390634FEFF0120003906388
:1008060050EFF0120003906351EFF07E197F201233
:100816003896EF4E6020120003906352EFF01200FC
:1008260003906353EFF0120003906354EFF012004D
:1008360003906355EFF07E197F26123896EF4E60CF
:100846002012000390633BEFF012000390633CEF2D
:10085600F012000390633DEFF012000390633EEF49
:10086600F07E197F2C123896EF4E6020120003900E
:100876006337EFF0120003906338EFF01200039035
:100886006339EFF012000390633AEFF0E4F527E4E2
:10089600F50DE5272401FFE433FE74372527F5829D
:1008A600E43463F583E0FD1240460527E527C3944B
:1008B6004340DCC2AFE4907FF0F0A3F0907FFD747C
:1008C600AAF0A374FFF0A37455F0E4F5A780FE7EAA
:0808D600637F767D081237886C
:0108DE0022F7
:103FB400AE07EEC39430400BEED394395005EE2493
:103FC400D0FF22EEC39461400BEED394665005EE0D
:103FD40024A9FF22EEC39441400BEED3944650052E
:083FE400EE24C9FF22AF062202
:104108009062ADE004F070069062ACE004F090625A
:0A411800ACE0FEA3E0FF1240B2226B
:10000300124108123FB4EFC454F0FEC00612410877
:08001300123FB4D0E02FFF22E0
:103E1400E4906B8BF0124108906B8CEFF0C39430FC
:103E24004018E0FFD394395011906B8BE02405F5D2
:103E340082E43461F583EFF08011906B8BE024050C
:103E4400F582E43461F583E4F0800C906B8BE0043C
:103E5400F0E0D3940840BE752D00752E00752F0038
:0C3E6400E4F5307B017A6179051227F348
:013E7000222F
:043896008E2A8F2BBC
:10389A009062ACE4F0A374FFF0124108EF606EF49A
:1038AA00606B852B82852A83E493B507EC752C011E
:1038BA00E52B252CF582E4352AF583E493602590DF
:1038CA0062ADE0252CFF9062ACE03400FE1240B2FB
:1038DA00E52B252CF582E4352AF583E493B5070414
:1038EA00052C80CCE52B252CF582E4352AF583E4DA
:1038FA009370A6E52C24FFFFE434FFFE9062ADE04E
:10390A002FF09062ACE03EF07E007F0122E4FEFFE1
:01391A00228A
:10328B007E197F32123896EF4E70037F01227E1922
:10329B007F35123896EF4E600C124108EF24D02484
:1032AB00FF920F8002D20F7E197F3B123896EF4EA2
:1032BB00600C124108EF24D0906682F08005E490F8
:1032CB006682F07E197F41123896EF4E600C1241E8
:1032DB0008EF24D090668EF08005E490668EF07E29
:1032EB00197F47123896EF4E600C124108EF24D02D
:1032FB0024FF92018002C2017E197F4D123896EF96
:10330B004E600C124108EF24D09062B4F08005E4BB
:10331B009062B4F090633F63A20190667C63A2015C
:10332B007F061226E530013B7E197F53123896EF4C
:10333B004E603012000390667CEFF0120003906633
:10334B007DEFF012000390667EEFF01200039066A3
:10335B007FEFF0120003906680EFF012000390668F
:06336B0081EFF07F00225B
:103F2700906577E0C3947C40027F0A906577E0FE56
:103F370004F074B52EF582E43462F583EFF0BF0A1E
:103F470027906577E0FF04F074B52FF582E43462BB
:103F5700F583E4F0906577E0FF12391B906577747D
:093F670008F09062B6E004F022BB
:103ECD009080007480F090633763A201F583F582D2
:103EDD0063A2017F081226E590633F63A2019080E3
:103EED008863A2017F0A1226E59080927407F0A3E1
:103EFD0074D0F0A37406F0906349E0FF9080B1F0A8
:103F0D009080E1EFF09080957455F0A3F0908000D3
:0A3F1D007401F090800974F0F022A6
:103C7A00908009E04410F09080A0E070609080A1EC
:103C8A007482F09080A874FFF0A3F0A3F0A3F07FF1
:103C9A00039080AEEFF0A374CBF09080007402F032
:103CAA00906B7F1222C500000000906B7FE090802D
:103CBA0040F0906B80E0908041F0906B81E09080C2
:103CCA0042F0906B82E0908043F0A3E4F0A3F0A36B
:0D3CDA00F0A3F0908018F0A3F0A3F0A3F089
:013CE70022BA
:103E7100908009E04440F09080D17482F07F0390FB
:103E810080DEEFF0A374CCF09080027402F0906BAE
:103E9100831222C500000000906B83E0908058F0EF
:103EA100906B84E0908059F0906B85E090805AF09F
:103EB100906B86E090805BF0A3E4F0A3F0A3F0A305
:0B3EC100F0908030F0A3F0A3F0A3F01D
:013ECC0022D3
:103AA200908009E04420F09080B8E0706C9080B97A
:103AB2007482F07F039080C6EFF07FCDA3EFF07F9A
:103AC200039080C4EFF0A374CDF09080C074FFF037
:103AD200A3F0A3F0A3F09080017402F0906B871220
:103AE20022C500000000906B87E090804CF0906B44
:103AF20088E090804DF0906B89E090804EF0906B62
:103B02008AE090804FF0A3E4F0A3F0A3F0A3F0903A
:093B12008024F0A3F0A3F0A3F05D
:013B1B002287
:1039A0008C258D26A907EAFDE975F018A424ACFF43
:1039B000E5F034808F82F583EDF0EBFDE975F018CA
:1039C000A4FFAEF024ACFBEE34808B82F583A3ED34
:1039D000F08526828C83E0FDEF24A8FFEE3480FE84
:1039E0008F82F583EDF08526828C83A3E08F828E13
:1039F00083A3F0852682852583A3A3E0FDE975F0E6
:103A000018A424A8FFE5F03480FE8F82F583A3A3D9
:103A1000EDF08526828C83A3A3A3E08F828E83A3FF
:043A2000A3A3F0224A
:063788008D2AAB07AA0622
:10378E00908000E030E5079065797401F022906B2F
:10379E007FE0FCA3E0FDA3E0FEA3E0F52E8E2D8DD1
:1037AE002C8C2BAE02AF038E838F8263A201E52D8C
:1037BE00540744C0F583852E8263A201AF2A1227D7
:1037CE0057E4FCFDFEE52E252AF52EEE352DF52DC2
:1037DE00ED352CF52CEC352BF52B908040E52BF0B0
:1037EE00A3E52CF0A3E52DF0A3E52EF09080007458
:1037FE0020F0AF2EAE2DAD2CAC2B906B7F1222B9DC
:01380E002297
:06380F008D25AB07AA069F
:10381500908002E030E5079065797403F022906BA3
:1038250083E0FCA3E0FDA3E0FEA3E0F5298E288D4F
:10383500278C26AE02AF038E838F8263A201E52813
:10384500540744D0F58385298263A201AF25122749
:1038550057E4FCFDFEE5292525F529EE3528F52853
:10386500ED3527F527EC3526F526908058E526F029
:10387500A3E527F0A3E528F0A3E529F090800274DD
:1038850020F0AF29AE28AD27AC26906B831222B964
:013895002210
:02352E008F25E7
:10353000908001E030E5099065797402F07F002207
:10354000906B87E0FCA3E0FDA3E0FEA3E0F5298EED
:10355000288D278C2690667C63A201E528540744B9
:10356000C8F58385298263A2017F0612276DE529AC
:103570002406F529E43528F528E43527F527E43530
:1035800026F52690657A63A201E528540744C8F51C
:103590008385298263A201AF2512276DE4FCFDFE1D
:1035A000E5292525F529EE3528F528ED3527F527D8
:1035B000EC3526F52690804CE526F0A3E527F0A310
:1035C000E528F0A3E529F09080017420F0AF29AE42
:0D35D00028AD27AC26906B871222B9AF25DD
:0135DD0022CB
:102FAF009081E0E0F5250525052505250525052555
:102FBF0005250525052505250525908010E0F52813
:102FCF00A3E0F529A3E0F52AA3E0F52B9081E1E03A
:102FDF00F5250525052505250525052505250525A2
:102FEF00052505250525908014E0F52CA3E0F52D8A
:102FFF00A3E0F52EA3E0F52FE52EB52A08E52FB5B2
:10300F002B037F0022E4F525E52E540744E0F583DA
:10301F00852F8263A20190637663A2017F08122736
:10302F009D90637863A2019062AE63A2017F061246
:10303F0026E5906376E0F526A3E0F527E4F52590E5
:10304F006376E0702AA3E024F8F525E52E540744B3
:10305F00E0F583852F8274082582F582E43583F5A8
:10306F008363A20190637663A201AF2512279DAE01
:10307F0026E4FCFDE52F2527F52FE52E3EF52EED59
:10308F00352DF52DEC352CF52C908014E52CF0A377
:10309F00E52DF0A3E52EF0A3E52FF090800074400E
:0330AF00F0AF255A
:0130B20022FB
:102997009081E6E0F525052505250525052505256D
:1029A70005250525052505250525908028E0F52819
:1029B700A3E0F529A3E0F52AA3E0F52B9081E7E052
:1029C700F5250525052505250525052505250525C0
:1029D70005250525052590802CE0F52CA3E0F52D90
:1029E700A3E0F52EA3E0F52FE4F525E52EB52A0A99
:1029F700E52FB52B05C208022B03E52E540744F03B
:102A0700F583852F8263A20190637663A2017F0815
:102A170012279D906376E0F526A3E0F527E5274585
:102A27002670099080027410F07F0022906683E080
:102A3700FFF46030906378E06F6003022ACA906603
:102A470084E0FF906379E06F7079906685E0FF908E
:102A5700637AE06F706D906686E0FF90637BE06F4E
:102A67006031805F906378E0906683F0906379E0EF
:102A7700906684F090637AE0906685F090637BE0DF
:102A8700906686F090637CE0FFA3E090634ACFF006
:102A9700A3EFF0906376E0702AA3E024F8F525E52C
:102AA7002E540744F0F583852F8274082582F5821A
:102AB700E43583F58363A20190637663A201AF25B2
:102AC70012279DAE26E4FCFDE52F2527F52FE52EE1
:102AD7003EF52EED352DF52DEC352CF52CAF2BAE27
:102AE7002AAD29AC28AB2FAA2EA92DA82CD31222A8
:102AF700A840099080027410F07F002290802CE596
:102B07002CF0A3E52DF0A3E52EF0A3E52FF09080A0
:062B1700027440F0AF253E
:012B1D002295
:102B1E009081E3E0F52505250525052505250525E7
:102B2E000525052505250525052590801CE0F5289C
:102B3E00A3E0F529A3E0F52AA3E0F52B9081E4E0CC
:102B4E00F525052505250525052505250525052537
:102B5E00052505250525908020E0F52CA3E0F52D13
:102B6E00A3E0F52EA3E0F52FE4F525E52EB52A0A10
:102B7E00E52FB52B05C209022C74E52E540744E847
:102B8E00F583852F8263A20190600463A2017F0EFC
:102B9E001227B3906004E0F526A3E0F52790600CB1
:102BAE00E0FFF4604A90667CE0FEEF6E7079A3E081
:102BBE00FF90600DE06F706F90667EE0FF90600E8C
:102BCE00E06F706390667FE0FF90600FE06F70576C
:102BDE00906680E0FF906010E06F704B906681E031
:102BEE00FF906011E06F703FE4906013F0800890EA
:102BFE00601374FFF0D2D9906004E0702AA3E02431
:102C0E00F2F525E52E540744E8F583852F82740EE0
:102C1E002582F582E43583F58363A2019060046317
:102C2E00A201AF251227B3AE26E4FCFDE52F252722
:102C3E00F52FE52E3EF52EED352DF52DEC352CF53B
:102C4E002CAF2BAE2AAD29AC28AB2FAA2EA92DA8BE
:102C5E002CD31222A85006E5274526700990800134
:102C6E007410F07F0022908020E52CF0A3E52DF06B
:102C7E00A3E52EF0A3E52FF09080017440F0AF2570
:012C8E002223
:0431A3008E2A8F2BB6
:1031A700908000E030E5079065797401F022906B1C
:1031B7007FE0FCA3E0FDA3E0FEA3E0F5318E308DB8
:1031C7002F8C2EE531FFE5305407FEE42FF52DEE69
:1031D70034C0F52C852D82F5837423F0052DE52D5C
:1031E7007002052C532CC7F582852C83740AF005D1
:1031F7002DE52D7002052C532CC790633F63A20168
:10320700852C83852D8263A2017F061227577406BA
:10321700252DF52DE4352CF52C852A83852B826306
:10322700A201852C83852D8263A20112273BE4FC32
:10323700FDFE906B7FE0F8A3E0F9A3E0FAA3E02F8F
:10324700FFEE3AFEED39FDEC38FCEF2408FFE43ED3
:10325700FEE43DFDE43CFC906B7F1222B9906B7F4E
:10326700E0908040F0906B80E0908041F0906B811F
:10327700E0908042F0906B82E0908043F090800075
:033287007420F0C0
:01328A002221
:0A2EA8008E2A8F2B8C2C8D2D8B2E83
:102EB200908000E030E5079065797401F022906B14
:102EC2007FE0FCA3E0FDA3E0FEA3E0F5348E338DAA
:102ED200328C31E534FFE5335407FEE42FF530EE52
:102EE20034C0F52F853082F5837423F00530E53048
:102EF2007002052F532FC7F582852F83740AF005C0
:102F020030E5307002052F532FC790633F63A20153
:102F1200852F8385308263A2017F061227577406AC
:102F22002530F530E4352FF52F852A83852B8263F2
:102F3200A201852F8385308263A20112273B8F3540
:102F4200EF2530F530E4352FF52FE52E6017852C6F
:102F520083852D8263A201852F8385308263A2013E
:102F6200AF2E122757E5352408252EF52EFFE4FC57
:102F7200FDFEE5342FF534EE3533F533ED3532F51C
:102F820032EC3531F531908040E531F0A3E532F095
:102F9200A3E533F0A3E534F09080007420F0AF3461
:0C2FA200AE33AD32AC31906B7F1222B91F
:012FAE002200
:02391B008F3FDC
:10391D00908000E030E5079065797401F022906B9E
:10392D007FE0FCA3E0FDA3E0FEA3E0F5438E428D16
:10393D00418C40E543FFE5425407FEE42FFFEE3492
:10394D00C09062B563A201F5838F8263A201AF3F80
:10395D00122757E4FCFDFEE543253FF543EE3542C6
:10396D00F542ED3541F541EC3540F540908040E5AF
:10397D0040F0A3E541F0A3E542F0A3E543F09080CC
:10398D00007420F0AF43AE42AD41AC40906B7F125E
:02399D0022B94D
:01399F002205
:063371008E2A8F2BAB0534
:10337700908000E030E5079065797401F022906B4A
:103387007FE0FCA3E0FDA3E0FEA3E0F5318E308DE6
:103397002F8C2EE531FFE5305407FEE42FF52DEE97
:1033A70034C0F52C852D82F5837423F0052DE52D8A
:1033B7007002052C532CC7F582852C83EBF0052D65
:1033C700E52D7002052C90633F63A201852C838550
:1033D7002D8263A2017F061227577406252DF52D2E
:1033E700E4352CF52C532CC7E52A852D82852C83B3
:1033F700F0052DE52D7002052C532CC7F582852C81
:1034070083E52BF0052DE52D7002052C532CC7E520
:1034170031240AF531E43530F530E4352FF52FE462
:10342700352EF52E908040E52EF0A3E52FF0A3E58D
:1034370030F0A3E531F09080007420F0AF31AE306A
:0A344700AD2FAC2E906B7F1222B95E
:013451002258
:103D5100908009E04480F09080E97441F07F0990FF
:103D610080F6EFF0A37464F09080037402F0908009
:103D710003E020E1F9906A7B1222C5000000009067
:103D81006A7BE0908064F0906A7CE0908065F090BE
:103D91006A7DE0908066F0906A7EE0908067F0A393
:103DA100E4F0A3F0A3F0A3F090803CF0A3F0A3F023
:023DB100A3F07D
:013DB30022ED
:103452009081E9E0F5280528052805280528052892
:1034620005280528052805280528908034E0F52937
:10347200A3E0F52AA3E0F52BA3E0F52C9081EAE086
:10348200F5280528052805280528052805280528E2
:10349200052805280528908038E0F52DA3E0F52EB3
:1034A200A3E0F52FA3E0F530E52FB52B08E530B505
:1034B2002C037F0022AF30AE2FAD2EAC2DAB2CAA49
:1034C2002BA92AA829D31222A8400AAF30AE2CEE8B
:1034D2009FF528800AAF30EFF404AE2C2EF528E5D4
:1034E2002F540744E0F58385308263A201906A7FFE
:1034F20063A201AF281227CBE4FCFDFEE5302528AC
:10350200F530EE352FF52FED352EF52EEC352DF568
:103512002D908038E52DF0A3E52EF0A3E52FF0A342
:0B352200E530F09080037440F0AF280B
:01352D00227B
:0230B3008F2864
:1030B5009080E8E0640660037FFF22906A7BE0FC75
:1030C500A3E0FDA3E0FEA3E0F52C8E2B8D2A8C2931
:1030D500E4FFFEFDFCAB2CAA2BA92AA829C31222CA
:1030E500A870609081F9E0F529906A7BE0FCA3E087
:1030F500FDA3E0FEA3E0FFE4FAF9F8EF2401FFEAFF
:103105003EFEE93DFDE83CFC906A7B1222B9906ADF
:103115007BE0FCA3E0FDA3E0FEA3E0FFE4F8EF24E1
:1031250001FFEA3EFEE93DFDE83CFC906A7B122288
:10313500B9908064E0F529A3E0F52AA3E0F52BA377
:10314500E0F52C906A7F63A201E52B540744D8F57E
:1031550083852C8263A201AF28122785E4FCFDFE3E
:10316500E52C2528F52CEE352BF52BED352AF52A02
:10317500EC3529F529908064E529F0A3E52AF0A32B
:10318500E52BF0A3E52CF09080037420F0AF2CAE76
:0D3195002BAD2AAC29906A7B1222B97F0075
:0131A200220A
:1040B200A2AF9210C2AF438E2075D2028F828E833E
:0C40C200E0FFE4F5D2538EDFA21092AFB5
:0140CE0022CF
:10404600E5D220E0FBA2AF9210C2AF43D2028F822C
:104056008E83EDF075D25063D250A21092AFE5D2A6
:0340660020E0FB5C
:014069002234
:103A2400E4FDED2401FFE433FE1240B274372DF5BA
:103A340082E43463F583EFF00DBD3FE6E4FDED244D
:103A44007FFFE433FE1240B2742D2DF582E434611D
:103A5400F583EFF0742D2DF582E43461F583E07085
:103A64001B742D2DF582E43461F5837420F0742EDB
:103A74002DF582E43461F583E4F080040DBD80BE4D
:103A8400E49061ACF0FDEDFF7E001240B274AD2D08
:0D3A9400F582E43461F583EFF00DBDFEE92D
:013AA1002202
:023FEC008B2A1E
:103FEE00A2AF9210C2AF85A22B53A2FE8E838F82F8
:103FFE0005A28C838D8274091227E1E52A53A2FE55
:10400E0043A2201227E353A2DF852BA2A21092AF68
:01401E00FFA2
:01401F00227E
:1040CF00A2AF9210C2AF8C838D82EF1227E143A271
:0C40DF00201227E353A2DFA21092AFFFD3
:0140EB0022B2
:02406A008F25A0
:10406C00A2AF9210C2AFE4F5838D8274061227E1E1
:10407C00E52543A2201227E353A2DFA21092AF7FC3
:01408C000132
:01408D002210
:02408E008F257C
:10409000A2AF9210C2AFE4F5838D82740A1227E1B9
:1040A000E52543A2201227E353A2DFA21092AF7F9F
:0140B000010E
:0140B10022EC
:10260A00A907E7FFA805EF93C3966008403B74FC4F
:10261A002FFF80F00F08EF93C3966008402B74FBDE
:10262A002FFF80E00F08EF93C3966008401B74FAEF
:10263A002FFF80D00F08EF93D3966008400B74F9F0
:10264A002FFF80C01F1F1F1F1FEF54FEF80303F741
:10265A00E893FC08E893FD08E893FE08E893FF2254
:10266A0009E993C39D6008402974FB29F980F1099F
:10267A00E993C39E6008401A74FA29F980E209E9CD
:10268A0093D39F6008400B74F929F980D31919195B
:10269A001919E9C313C313FF22740093F8ECC39802
:1026AA004024701F740193F8EDC398401970147494
:0E26BA000293F8EEC398400E7009740393F873
:1026C800EFC39840037F00227F0122EDF8E6F0086F
:1026D800A3DFFA22EDF8E0F608A3DFFA22E0A3630D
:1026E800A201F0A363A201DFF475A2002263A20194
:1026F800F0A363A20122E0A363A201F0A363A201F5
:10270800E0A363A201F0A363A201E463A201F0A322
:1027180063A201DFE175A20022E0A363A2016DFEBE
:10272800936CFDEE058393FC158363A201DFEA75C4
:10273800A200227F00E493A363A201F00F600CA320
:10274800E583C2E3F58363A20180EA75A20022E073
:10275800A363A201F0A3E583C2E3F58363A201DFCB
:10276800EE75A20022E0A363A201F0A3E583C2E410
:10277800D2E3F58363A201DFEC75A20022E0A36334
:10278800A201F0A3E58344F8C2E5F58363A201DF63
:10279800EC75A20022E583C2E3F583E0A363A201FE
:1027A800F0A363A201DFEE75A20022E583C2E4D2A2
:0A27B800E3F583E0A363A201F0A3A0
:1027C20063A201DFEC75A20022E58344F8F583E001
:1027D200A363A201F0A363A201DFEE75A20022F9B6
:1027E20022C002C004C00612FFF0D006D004D002FC
:0127F20022C4
:101959003E2A2C312CCFE0F0E0ECE5F2F0FB20F848
:10196900E8EDFB2043414E0A003E4C2C6B30312CF4
:1019790025732C43EAEEF0EEF1F2FC20EDE020F8BD
:10198900E8EDE52043414E2C30202D20353030EA5A
:10199900E1283530EC292C31202D203530EAE12899
:1019A900353030EC290A0030202D20353030EAE17D
:1019B900283530EC290031202D203530EAE1283551
:1019C9003030EC29003E2A2C312CCFE0F0E0ECE558
:1019D900F2F0FB20EFF0EEF2EEEAEEEBE0204D4FF5
:1019E900444255530A003E4C2C4930312C256C7524
:1019F9002CD1EAEEF0EEF1F2FC20EEE1ECE5EDE0BF
:101A09002C343830302C393630302C3139323030B2
:101A19000A003E532C4931322C2562752CC0E4F062
:101A2900E5F120E1EBEEEAE020D2C8D220EDE0209A
:101A3900F8E8EDE50A003E532C6D2562752C256208
:101A4900752D25752D2562752D2562752CC7E0EF3D
:101A5900F0EEF1202562752028B9CFF02DD0E5E30D
:101A69002DCAEEEB2DD2E8EF290A003E532C563051
:101A7900382C25752CCFE0F3E7E020E220EEEFF0DB
:101A8900EEF1E0F528ECF1290A003C21003C6B302D
:101A9900313D003C4930313D003C4931323D003C4B
:101AA9005630383D002043616E4572474954002045
:101AB9000A002043616E457272434821000A0049B9
:101AC9006E69745443500A004C697374656E5443CB
:101AD900500A00534F434B5F5443505F45535441A1
:101AE900424C49534845440A000A2D3E20000A3C0D
:101AF9002D200020CEF2E2E5F23A00CEF8E8E1EA44
:101B0900E020CAD12100CEF8E8E1EAE020E0E4F0E3
:101B1900E5F1E02100CEF8E8E1EAE020F2E8EFE0C3
:101B29002100C7E0EFE8F1FC204F4B00CEF8E8E1D7
:101B3900EAE020E4EBE8EDFB21000AC7E0EFF0EE74
:101B4900F13A003C6D303D000000003C6D313D0034
:101B59000000003C6D323D000000003C6D333D004B
:101B69000000003C6D343D000000003C6D353D0037
:101B79000000003C6D363D000000003C6D373D0023
:101B89000000003C6D383D000000003C6D393D000F
:101B99000000003C6D31303D0000003C6D31313DAD
:101BA9000000003C6D31323D0000003C6D31333D99
:101BB9000000003C6D31343D0000003C6D31353D85
:101BC90000000000C1814001C0804101C080410086
:101BD900C1814001C0804100C1814000C1814001F3
:101BE900C0804101C0804100C1814000C1814001E4
:101BF900C0804100C1814001C0804101C0804100D5
:101C0900C1814001C0804100C1814000C1814001C2
:101C1900C0804100C1814001C0804101C0804100B4
:101C2900C1814000C1814001C0804101C0804100A3
:101C3900C1814001C0804100C1814000C181400192
:101C4900C0804101C0804100C1814000C181400183
:101C5900C0804100C1814001C0804101C080410074
:101C6900C1814000C1814001C0804101C080410063
:101C7900C1814001C0804100C1814000C181400152
:101C8900C0804100C1814001C0804101C080410044
:101C9900C1814001C0804100C1814000C181400132
:101CA900C0804101C0804100C1814000C181400123
:101CB900C0804100C1814001C0804101C080410014
:101CC900C1814000C0C101C30302C2C60607C705DE
:101CD900C5C404CC0C0DCD0FCFCE0E0ACACB0BC98F
:101CE9000908C8D81819D91BDBDA1A1EDEDF1FDD6F
:101CF9001D1CDC14D4D515D71716D6D21213D3113F
:101D0900D1D010F03031F133F3F23236F6F737F53E
:101D19003534F43CFCFD3DFF3F3EFEFA3A3BFB39CE
:101D2900F9F83828E8E929EB2B2AEAEE2E2FEF2DCE
:101D3900EDEC2CE42425E527E7E62622E2E323E17E
:101D49002120E0A06061A163A3A26266A6A767A59E
:101D59006564A46CACAD6DAF6F6EAEAA6A6BAB690E
:101D6900A9A86878B8B979BB7B7ABABE7E7FBF7DEE
:101D7900BDBC7CB47475B577B7B67672B2B373B1BE
:101D89007170B050909151935352929656579755FE
:101D99009594549C5C5D9D5F9F9E5E5A9A9B5B994E
:101DA900595898884849894B8B8A4A4E8E8F4F8D4E
:101DB9004D4C8C44848545874746868242438341FE
:031DC900818040D6
:1040F2005266900000000000000000000000000076
:054102000000000000B8
:014135002267
:03002300023B9607
:103B9600C0E0C083C082C0D075D01830982CE556DE
:103BA60025E9F5EB30D709E55525F904F5FB80063F
:103BB600E55525F9F5FBD29174592558F582E4347B
:103BC60069F583E599F00558C29830992DE559C3F2
:103BD60095575015D290AF59055974592FF582E46F
:103BE600346AF583E0F599800FAF578F59EF600877
:103BF600C2190559D296C290C299D0D0D082D0832C
:033C0600D0E032D9
:10402000C2A9438902758C48758A4875D90475DB25
:104030004875DC4875DD4875DE48E4F5E9F5F9C2F8
:06404000D9D28CD2DE2271
:102D9C007BFF7A197959121E2E9068B2E070147567
:102DAC002EFF752F197530B07BFF7A197972121EB0
:102DBC002E8012752EFF752F197530BF7BFF7A1977
:102DCC007972121E2E7BFF7A1979CE121E2E906A02
:102DDC0079E0FEA3E0FFC3E49FFFE49EFEAB07FA9D
:102DEC003395E0F9F87F007E8C7D0A7C0012220876
:102DFC008F318E308D2F8C2E7BFF7A1979EF121E2E
:102E0C002E7BFF7A1A791B9068B3E0F52E121E2EDA
:102E1C00E4F52A7BFF7A1A793F852A2EE52AFD33C1
:102E2C0095E0FC74C62DF58274683CF583E0F52FB3
:102E3C00AF2AEF3395E0FEEF25E0FFEE33FE74D7BB
:102E4C002FF58274683EF583E0F530A3E0F531741C
:102E5C00F72DF58274683CF583E0F532AF2AEF3339
:102E6C0095E0FE74082FF58274693EF583E0F53326
:102E7C00E52A04F534121E2E052AC3E52A64809433
:102E8C00904090AE5DAF5E7C007D0A1221288E2EA4
:0B2E9C008F2F7BFF7A1A7974121E2E14
:012EA7002208
:1023EE007E1A7F93123896EF4E70037F0122E4908F
:1023FE0068B2F07E1A7F96123896EF4E601B12412D
:10240E00088F25E525B431069068B2740AF0E525EB
:10241E00B432069068B27464F07E1A7F9C123896BD
:10242E00EF4E600D123E148F298E288D278C26803C
:10243E000BE4752980752825F527F526AB29AA28E2
:10244E00A927A8267F007E8C7D0A7C001222081206
:10245E00229A906A79EEF0A3EFF0E47B64FAF9F831
:10246E00AF29AE28AD27AC26122208A804A905AACA
:10247E0006AB07E47F587E1BFDFC1222088E558F9B
:10248E00567E1A7FA2123896EF4E600A123E1490B4
:10249E0068B3EFF08005E49068B3F07E1A7FA8125F
:1024AE003896EF4E6012123E14E47B0AFAF9F812D7
:1024BE00217D8E5D8F5E8006755D01755EF4E4F59F
:1024CE0054F525E525FD3395E0FC74C62DF5827493
:1024DE00683CF583E4F0E525FB3395E0FAEB25E067
:1024EE00FFEA33FE74D72FF58274683EF583E4F06D
:1024FE00A3F074F72DF58274683CF583E4F0AF25F4
:10250E00EF3395E0FE74082FF58274693EF583E48F
:10251E00F074B42FF58274683EF583E4F074A22F44
:10252E00F58274683EF583740FF0EBAE027803C348
:10253E0033CE33CED8F9244CF582741B3EAF82FED7
:10254E00123896EF4E70030225F6123E14E525FD65
:10255E003395E0FC74C62DF58274683CF583EFF07C
:10256E0074C62DF58274683CF583E0607B123E14D0
:10257E00AD07AC06AF25EF3395E0FEEF25E0FFEE9D
:10258E0033FE74D72FF58274683EF583ECF0A3ED1D
:10259E00F0123E14E525FD3395E0FC74F72DF5821F
:1025AE0074683CF583EFF0123E14E525FD3395E09B
:1025BE00FC74082DF58274693CF583EFF074B42D2C
:1025CE00F58274683CF583E554F074082DF5827439
:1025DE00693CF583E06406600F74F72DF58274682C
:1025EE003CF583E02554F5540525C3E52564809418
:0B25FE009050030224D17554FF7F00B1
:0126090022AE
:103CE80043AB01C2E8C2EAE4FFEFC454F0F5B1C344
:103CF800EF64809488500575B3D08003E4F5B3E48D
:103D0800F5B275BCC8F5BDF5BE75BF7875C4FFF5CD
:103D1800C5F5C675C778F5A3F5A3F5A3F5A3F5A36F
:103D2800F5A3F5A3F5A30FBF0EBF9068B2E0FF257A
:103D3800E0F5B475B50C75B66C75A11275AB027566
:083D4800C13E75C3FF75C20303
:013D50002250
:103DB40075B180E4F5B3F5B28545BCE5465403FF1F
:103DC40033333354F8FFE54654E04FFFE547C4135B
:103DD40054074FF5BDE54733333354F8FFE548C482
:103DE4001354074FF5BEE54833333354F8F5BF8514
:103DF4004AA3854BA3854CA3854DA3854EA3854F2C
:103E0400A38550A38551A3E549540F2450F5B3224B
:102C8F00E59B541F6020200B1A7E1A7FAE1231A3D2
:102C9F00E59B541FFF7E007D031233717E1A7FB8B0
:102CAF001231A3E4F59BE5BA30E008E4F5B375B152
:102CBF0080F5B2E5CFF47003022D99752901E4F583
:102CCF0028E5CFF455297003022D87E528C454F069
:102CDF00F5B1E5B2547F6420706FE5B3540FF54939
:102CEF0085BC45E5BD541FFF131313541FFFE5BDEE
:102CFF0054E044184FF546E5BDC43354E0FFE5BE3C
:102D0F00131313541F4FF547E5BEC43354E0FFE5CB
:102D1F00BF131313541F4FF54885A34A85A34B8543
:102D2F00A34C85A34D85A34E85A34F85A35085A3A3
:102D3F0051E4F5B2E545547EB5450575B3508003B2
:102D4F0075B3D0E5492405FF22E5B2549F602320D7
:102D5F000B207E1A7FBB1231A3AFB27E007D031210
:102D6F003371AFB37E007D031233717E1A7FC612AB
:102D7F0031A3E4F5B275B3D0E52925E0F52905288F
:0C2D8F00E528C394085003022CD07F00FC
:012D9B002215
:103B1C00C219E4F558F50BD296F557F559FF7F40CD
:103B2C00906919E4F0A3DFFC7F40E4F55AF55C12D0
:103B3C0023EE123CE8C2ADE4F5C9D2CDD2CCC2C959
:103B4C00C2CAF5CDF5CC906A79E0F5CBA3E0F5CA05
:103B5C0085CBCD85CACCE4F598D29E438740C29FD5
:103B6C00C2ACC298C29975B81075B710D2CAD29CA3
:103B7C00D2AC124020C2D9E5E92464F5EB30D7066B
:093B8C00E5F904F5FB2285F9FBC3
:013B9500220D
:014136002266
:014137002265
:05001E00D29CD2AC22CF
:014138002264
:063F7000AC05AB07AA0638
:103F760090690774FFF0906918F0AF041CEF602D8C
:103F86000BEBAE0270010A14F5828E83E0FF906996
:103F960007E06FFF901BCC93FE906918E06E906966
:0D3FA60007F0EF901CCC93906918F080CDCF
:013FB30022EB
:103C090074C62554F582E43468F583E0906A59F066
:103C190074082554F582E43469F583E0906A5AF012
:103C2900E55425E024D7F582E43468F583E0FCA364
:103C3900E0FDEC906A5BF0A3EDF0E4A3F074F725E6
:103C490054F582E43468F583E0906A5EF07E6A7F19
:103C5900597D06123F70906907E0906A5FF090699C
:103C690018E0906A60F0E4F559755708C296D29940
:013C79002228
:10366E00E55CC394404003E4F55C7419255CF58277
:10367E00E43469F583E0FF30E16F7419255CF5825F
:10368E00E43469F583EF54FDF0E4906476F0A374AE
:10369E000DF090667BE0906478F0A37419F0A3743B
:1036AE0048F0A37479F0E55C131313541FFF906870
:1036BE00B3E02F90647CF0E55C540725E025E02410
:1036CE0080A3F0A37408F0F5F0E55CA424A2F582C3
:1036DE00E5F03466F58363A20190647F63A2017FF7
:0E36EE00081226E5055C7F0122055C7F0022A4
:014139002263
:100F67003000469080E8E0700F123D51300D077E4B
:100F77001A7FC81231A3C21B9080E8E0B40E12900A
:100F870080037408F0300D077E1A7FD11231A3C297
:100F97001B9080E8E0B4060F201B0C300D077E1A6B
:100FA7007FDC1231A3D21BC200201B030210692071
:100FB70019071234528F258003E4F525E52560478C
:100FC700300D0C7E1A7FF27C6A7D7FFB122EA8E51E
:100FD700E92410F5EB30D708E5F92428F5FB80065E
:100FE700E5F92427F5FB906A7F63A201906A5963AC
:100FF700A201AF251226E5852557E4F559D290C2FF
:1010070091D219C296D29920D9030214C7C2D9E541
:10101700E92410F5EB30D708E5F92428F5FB80061D
:10102700E5F92427F5FBE558D3940050030214C7CC
:10103700C29185585BE4F55890695963A201906A9B
:101047007F63A201AF5B1226E5AF5B1230B3200DC1
:10105700030214C77E1A7FF77C6A7D7FAB5B122E73
:10106700A8227419255AF582E43469F583E020E053
:1010770002055AE55AC394404003E4F55A122C8FEF
:10108700EF606BE548640F70659068B3E0FF6547F4
:10109700705C7419255AF582E43469F583E0FE30F3
:1010A700E04C7419255AF582E43469F583EE54FE51
:1010B700F0754548754679E55A131313541FFEEF2B
:1010C7002EF547E55A540725E025E02480F54875B5
:1010D700490875F008E55AA424A2F582E5F03466BC
:1010E700F5837D4A7F081226DC123DB4055A30028B
:1010F70049C2029068C5E004F070069068C4E00435
:10110700F0D39068C5E094B89068C4E0940B402A87
:10111700E4F0A3F0F52574192525F582E43469F583
:1011270083E030E20E74192525F582E43469F583EE
:101137007403F00525E525B440DC20D9030214C764
:10114700E5577003021450E558D394005003021377
:1011570027C29185585B74B42554F582E43468F549
:1011670083E075F002A485F026F527E4F5587E693B
:101177007F59AD5B123F70200B0D7E1A7FFC7C6997
:101187007D59AB5B122EA8906918E0FF906907E0C4
:101197004F6010300B030214507E1B7F041231A3E3
:1011A70002145074C62554F582E43468F583E0FFD1
:1011B700906959E06F6010300B030214507E1B7F5B
:1011C7000F1231A302145074082554F582E43469D0
:1011D700F583E0FF90695AE06F6010300B0302144B
:1011E700507E1B7F1E1231A302145090695AE0B43F
:1011F7000610300B030214507E1B7F2B1231A30203
:10120700145074F72554F582E43468F583E075F0DB
:1012170002A4FF90695BE06F7002E5F06010300B8D
:10122700030214507E1B7F351231A302145074A29F
:101237002554F582E43468F583E4F0F52590695B7D
:10124700E0FFE525C39F400302145074A22527F54C
:101257008274663526F583E0FF745D2525F582E403
:101267003469F583E0FEEF6E602774A22527F582C7
:1012770074663526F583EEF0E527AE267803CEC3F0
:1012870013CE13D8F92419F58274693EF5837407D0
:10129700F0E527AE267803CEC313CE13D8F9241969
:1012A700F58274693EF583E04404F00527E527706D
:1012B70002052624A2F58274663526F583E0FF74BD
:1012C7005C2525F582E43469F583E0FEEF6E60273F
:1012D70074A22527F58274663526F583EEF0E52797
:1012E700AE267803CEC313CE13D8F92419F582742A
:1012F700693EF5837407F0E527AE267803CEC3135E
:10130700CE13D8F92419F58274693EF583E04404B5
:10131700F00527E527700205260525052502124455
:1013270074082554F582E43469F583E06406700394
:1013370002145074A22554F582E43468F583E0045E
:10134700F074A22554F582E43468F583E0D3940A57
:10135700500302145074A22554F582E43468F583CF
:101367007405F074B42554F582E43468F583E075A8
:10137700F002A485F026F527E4F52574F72554F542
:1013870082E43468F583E0FFE525C39F4003021438
:101397005074A22527F58274663526F583E0F4603C
:1013A7002874A22527F58274663526F58374FFF025
:1013B700E527AE267803CEC313CE13D8F92419F543
:1013C7008274693EF5837407F0E527AE267803CE6D
:1013D700C313CE13D8F92419F58274693EF583E057
:1013E7004404F00527E5277002052624A2F5827438
:1013F700663526F583E0647F602874A22527F58289
:1014070074663526F583747FF0E527AE267803CE1C
:10141700C313CE13D8F92419F58274693EF5837482
:1014270007F0E527AE267803CEC313CE13D8F924E9
:1014370019F58274693EF583E04404F00527E52732
:101447007002052605250213820554E4F557E55475
:10145700C39410504974C62554F582E43468F58363
:10146700E0605D74F72554F582E43468F583E06045
:101477004FC2D9123C09E5E924E8F5EB30D708E576
:10148700F92404F5FB8006E5F92403F5FB200B306E
:101497007E1B7F437C6A7D597B08122EA8227554D8
:1014A700FFE55E455D6019C2D9E55E25E9F5EB30DC
:1014B700D708E55D25F904F5FB22E55D25F9F5FB80
:0114C7002202
:034132007F0022E9
:103708000208DFE493A3F8E493A34003F68001F2F0
:1037180008DFF48029E493A3F85407240CC8C333C2
:10372800C4540F4420C8834004F456800146F6DF91
:10373800E4800B01020408102040809040ECE47EF5
:10374800019360BCA3FF543F30E509541FFEE49386
:10375800A360010ECF54C025E060A840B8E493A34D
:10376800FAE493A3F8E493A3C8C582C8CAC583CA78
:10377800F0A3C8C582C8CAC583CADFE9DEE780BE30
:0141070000B7
:10212800BC000BBE0029EF8DF084FFADF022E4CC9B
:10213800F875F008EF2FFFEE33FEEC33FCEE9DEC64
:10214800984005FCEE9DFE0FD5F0E9E4CEFD22EDAA
:10215800F8F5F0EE8420D21CFEADF075F008EF2FF4
:10216800FFED33FD4007985006D5F0F222C398FDE5
:052178000FD5F0EA2282
:10217D00E88FF0A4CC8BF0A42CFCE98EF0A42CFC01
:10218D008AF0EDA42CFCEA8EF0A4CDA8F08BF0A47F
:10219D002DCC3825F0FDE98FF0A42CCD35F0FCEBDE
:1021AD008EF0A4FEA9F0EB8FF0A4CFC5F02ECD39A3
:0F21BD00FEE43CFCEAA42DCE35F0FDE43CFC2210
:1021CC0075F008758200EF2FFFEE33FECD33CDCCCA
:1021DC0033CCC58233C5829BED9AEC99E58298404D
:1021EC000CF582EE9BFEED9AFDEC99FC0FD5F0D62A
:1021FC00E4CEFBE4CDFAE4CCF9A88222B800C1B954
:10220C000059BA002DEC8BF084CFCECDFCE5F0CB91
:10221C00F97818EF2FFFEE33FEED33FDEC33FCEBCA
:10222C0033FB10D703994004EB99FB0FD8E5E4F985
:10223C00FA227818EF2FFFEE33FEED33FDEC33FC72
:10224C00C933C910D7059BE99A4007EC9BFCE99A66
:10225C00F90FD8E0E4C9FAE4CCFB2275F010EF2FAB
:10226C00FFEE33FEED33FDCC33CCC833C810D707AB
:10227C009BEC9AE899400AED9BFDEC9AFCE899F8E6
:0E228C000FD5F0DAE4CDFBE4CCFAE4C8F92279
:0E229A00C3E49FFFE49EFEE49DFDE49CFC2255
:1022A800EB9FF5F0EA9E42F0E99D42F0E89C45F08C
:0122B8002203
:0C22B900ECF0A3EDF0A3EEF0A3EFF02298
:1022C500A8828583F0D083D0821222DC1222DC1210
:1022D50022DC1222DCE473E493A3C583C5F0C58335
:1022E500C8C582C8F0A3C583C5F0C583C8C582C863
:0122F50022C6
:101DCC00E53A242EF8E6053A22782B301702782EC5
:101DDC00E475F00112234E0222F62010EB7F2ED276
:101DEC00108018EF540F2490D43440D4FF30140BCF
:101DFC00EF24BFB41A0050032461FFE53B600215C9
:101E0C003B053EE53E7002053D30170D782BE47521
:101E1C00F00112234EEF02233C023F277403D2172A
:101E2C008003E4C217F53A8B2B8A2C892DE4F53B01
:101E3C00F53DF53EE53B60077F20121E0780F575EA
:101E4C003CFFC211C210C212C213C215C216C21874
:101E5C00121DD5FF700D3017057F00121E18AF3EF6
:101E6C00AE3D22B4255FC2D5C214121DD5FF24D0BD
:101E7C00B40A00501A75F00A783B30D50508B6FF45
:101E8C000106C6A426F620D5047002D21380D924EC
:101E9C00CFB41A00EF5004C2E5D214022018D211AC
:101EAC0080C6D21080C0D21280BCD2D580BAD215D6
:101EBC0080B47F20121E072012077401B53B00402E
:101ECC00F1121DCCFF121E07021E40D218D2168032
:101EDC0095121DCCFB121DCCFA121DCCF94A4B707D
:101EEC000679E97A207BFF20122EE53B602A7E00E2
:101EFC008E8275830012230F60060EEE653C70F027
:101F0C00C2D5EBC0E0EAC0E0E9C0E0EE12205FD041
:101F1C00E0F9D0E0FAD0E0FB1222F6FF60AAEBC0A9
:101F2C00E0EAC0E0E9C0E0121E07D0E02401F9D0DD
:101F3C00E03400FAD0E0FBE53C0460DCD53CD98011
:101F4C00877BFF7A20795BD212809C791080027992
:101F5C0008C216C2188008D2D5790A8004790AC240
:101F6C00D5E53C047002F53CE4FAFDFEFF121DCCF5
:101F7C00FC7B08201113121DCCFD7B1030100A12B3
:101F8C001DCCFE121DCCFF7B20EC3382D592D5509C
:101F9C0013C3E43010069FFFE49EFEE42011039D62
:101FAC00FDE49CFCE4CBF8C211EC700CCFCECDCC94
:101FBC00E824F8F870F38017C3EF33FFEE33FEED2F
:101FCC0033FDEC33FCEB33FB994002FB0FD8E9EB10
:101FDC00301105F8D0E0C448B211C0E00AEC4D4E07
:101FEC004F78207B0070C2EAB53C0040BCC0E012C8
:101FFC002061D0F0D0E0201104C4C0E0C4B211C004
:10200C00F0121DF0D0F0D5F0EB021E401223AD1EE5
:10201C00DD531F57581EAE4C1EAA421F5B4F1F6349
:0F202C00441F63491EC3431F69551F4D461F4D77
:10203B00451F4D472109501EB22D1EB62E1ED92B02
:10204B001EBA231ED72020F22A1E724800001ED172
:10205B003F3F3F00790AA2D5201314301509B91060
:10206B00020404B9080104A2D52016025001042071
:10207B0012689212B53B005034C0E07F2030131928
:10208B007F30A21272167215500F1220B8C212C2F4
:10209B0016C215C2187F30800F301503E9C0E0124D
:1020AB001E07301503D0E0F9D0E0B53BCC30151747
:1020BB007F30B9100C121E077F583014077F7880C1
:1020CB0003B90803121E073012057F2D021E077F6E
:1020DB00202018F87F2B2016F322921280CF286E27
:1020EB00756C6C2900D211121DCC3011F8C211780D
:1020FB003B30D50108F6021E722D50434958121D74
:10210B00CC2403B405004001E490210493121DF884
:0D211B00743A121DF8D213753B04021F57D1
:1027F3008B2A8A2B892CE4F536F535F534F533F538
:1028030031F532E52E452F452D6012EBC0E0EAC0CD
:10281300E0E9C0E0AB2DAA2EA92F12235EAB2A0557
:102823002CE52CAA2B7002052B14F91222F6F5378E
:10283300C394094007E537D3940D40E1E53764209D
:1028430060DBE537B42D054332038016E537B42B3F
:1028530005433201800C74FF252CF52C74FF352BB6
:10286300F52BE53060046410703FAB2AAA2BA92C2A
:102873001222F664306009E530702E75300A802923
:1028830090000112230FFF64786004EFB4581343E0
:1028930032017530107402252CF52CE4352BF52B01
:1028A3008007E5307003753008AB2A052CE52CAAA8
:1028B3002B7002052B14F91222F6F537C3946140ED
:1028C3000AE537D3947A50035337DF74D02537F5AD
:1028D30037C3940A400CE5379411406D74F92537DA
:1028E300F537E537D39530506043320185363B8564
:1028F300353A853439853338AF307E00E4FCFDAB9F
:1029030036AA35A934A83312217DC8ECC8C9EDC94C
:10291300CAEECACBEFCBE4FCFDFEEB2537F536EE72
:102923003AF535ED39F534EC38F533AF36AE35AD30
:1029330034FCAB3BAA3AA939A838D31222A85003D6
:102943000228AC4332040228ACE53220E003E480E1
:102953002DE52E452F452D601EAB2AE52C24FFF9CE
:10296300E52B34FFFAEBC0E0EAC0E0E9C0E0AB2DB1
:10297300AA2EA92F12235EE53230E20774FFFFFE71
:10298300FDFC22E532AF36AE35AD34AC3330E10376
:0429930002229A2260
:1022F600BB010689828A83E0225002E722BBFE02E6
:09230600E32289828A83E4932218
:10230F00BB010CE58229F582E5833AF583E0225083
:10231F0006E92582F8E622BBFE06E92582F8E222CD
:0D232F00E58229F582E5833AF583E49322E7
:10233C00BB010689828A83F0225002F722BBFE0180
:02234C00F3227A
:10234E00FAE6FB0808E6F925F0F618E6CA3AF62290
:10235E00BB011A89828A83D0F0D0E0F8D0E0F9D0A0
:10236E00E0FAD0E0FBE8C0E0C0F00223DC5016E952
:10237E00F8D083D082D0E0F9D0E0FAD0E0FBC08272
:10238E00C0830223D3BBFE16E9F8D083D082D0E0FF
:0F239E00F9D0E0FAD0E0FBC082C0830223E52231
:1023AD00D083D082F8E4937012740193700DA3A3BF
:1023BD0093F8740193F5828883E4737402936860D3
:0623CD00EFA3A3A380DFD3
:0923D300EBF608EAF608E9F6222F
:0923DC00EBF0A3EAF0A3E9F02202
:0923E500EBF208EAF208E9F22229
:00000001FF
